ARM Linker, RVCT3.1 [Build 942] for uVision [Standard]

================================================================================

Section Cross References

    startup_mps.o(STACK) refers (Special) to stkheap2.o(.text) for __use_two_region_memory
    startup_mps.o(HEAP) refers (Special) to stkheap2.o(.text) for __use_two_region_memory
    startup_mps.o(RESET) refers to startup_mps.o(STACK) for __initial_sp
    startup_mps.o(RESET) refers to startup_mps.o(.text) for Reset_Handler
    startup_mps.o(RESET) refers (Special) to stkheap2.o(.text) for __use_two_region_memory
    startup_mps.o(.text) refers to __main.o(!!!main) for __main
    startup_mps.o(.text) refers to startup_mps.o(HEAP) for Heap_Mem
    startup_mps.o(.text) refers to startup_mps.o(STACK) for Stack_Mem
    startup_mps.o(.text) refers (Special) to stkheap2.o(.text) for __use_two_region_memory
    stkheap2.o(.text) refers to sys_stackheap_outer.o(.text) for __user_setup_stackheap
    stkheap2.o(.text) refers to rt_stackheap_storage_intlibspace.o(.text) for __rt_stackheap_storage
    __main.o(!!!main) refers to kernel.o(.text) for __rt_entry
    kernel.o(.text) refers to stkheap2.o(.text) for __rt_stackheap_init
    kernel.o(.text) refers to boardinit2.o(.text) for _platform_post_stackheap_init
    kernel.o(.text) refers to lib_init.o(.text) for __rt_lib_init
    kernel.o(.text) refers to boardinit3.o(.text) for _platform_post_lib_init
    kernel.o(.text) refers to main.o(.text) for main
    kernel.o(.text) refers to exit.o(.text) for exit
    kernel.o(.text) refers to sys_exit.o(.text) for _sys_exit
    kernel.o(.ARM.exidx) refers to kernel.o(.text) for __rt_entry
    sys_stackheap_outer.o(.text) refers to libspace.o(.text) for __user_perproc_libspace
    sys_stackheap_outer.o(.text) refers to startup_mps.o(.text) for __user_initial_stackheap
    rt_stackheap_storage.o(.text) refers to rt_stackheap_storage.o(.bss) for __rt_stackheap_storage_data
    rt_stackheap_storage_intlibspace.o(.text) refers to libspace.o(.bss) for __libspace_start
    sys_exit.o(.text) refers to use_no_semi.o(.text) for __I_use_semihosting
    libspace.o(.text) refers to libspace.o(.bss) for __libspace_start
    exit.o(.text) refers to kernel.o(.text) for __rt_exit
    stkheap1.o(.text) refers to sys_stackheap_outer.o(.text) for __user_setup_stackheap
    stkheap1.o(.text) refers to rt_stackheap_storage_intlibspace.o(.text) for __rt_stackheap_storage
    lib_init.o(.emb_text) refers to no_argv.o(.text) for __ARM_get_argv
    lib_init.o(.text) refers to fpinit.o(x$fpl$fpinit) for _fp_init
    lib_init.o(.text) refers to lib_init.o(.emb_text) for __ARM_argv_veneer
    lib_init.o(.text) refers to rt_locale_intlibspace.o(.text) for __rt_locale
    rt_locale.o(.text) refers to rt_locale.o(.bss) for __rt_locale_data
    rt_locale_intlibspace.o(.text) refers to libspace.o(.bss) for __libspace_start
    _get_argv.o(.text) refers to heapext.o(.text) for __heap_extend
    _get_argv.o(.text) refers to defsig_rtmem_outer.o(.text) for __rt_SIGRTMEM
    _get_argv.o(.text) refers to sys_command.o(.text) for _sys_command_string
    _get_argv.o(.text) refers (Special) to hrguard.o(.text) for __heap_region_guard
    fpinit.o(x$fpl$fpinit) refers to rt_fp_status_addr_intlibspace.o(.text) for __rt_fp_status_addr
    sys_command.o(.text) refers (Special) to use_no_semi.o(.text) for __I_use_semihosting
    rt_fp_status_addr.o(.text) refers to rt_fp_status_addr.o(.bss) for __rt_fp_status_addr_data
    rt_fp_status_addr_intlibspace.o(.text) refers to libspace.o(.bss) for __libspace_start
    defsig_rtmem_outer.o(.text) refers to defsig_rtmem_inner.o(.text) for __rt_SIGRTMEM_inner
    defsig_rtmem_outer.o(.text) refers to defsig_exit.o(.text) for __sig_exit
    defsig_rtmem_formal.o(.text) refers to rt_raise.o(.text) for __rt_raise
    heapext.o(.text) refers to stkheap2.o(.text) for __rt_heap_extend
    rt_raise.o(.text) refers to __raise.o(.text) for __raise
    rt_raise.o(.text) refers to sys_exit.o(.text) for _sys_exit
    defsig_exit.o(.text) refers to sys_exit.o(.text) for _sys_exit
    defsig_rtmem_inner.o(.text) refers to defsig_general.o(.text) for __default_signal_display
    __raise.o(.text) refers to defsig.o(CL$$defsig) for __default_signal_handler
    defsig_general.o(.text) refers to sys_wrch.o(.text) for _ttywrch
    sys_wrch.o(.text) refers (Special) to use_no_semi.o(.text) for __I_use_semihosting
    defsig.o(CL$$defsig) refers to defsig_rtmem_inner.o(.text) for __rt_SIGRTMEM_inner
    defsig_abrt_inner.o(.text) refers to defsig_general.o(.text) for __default_signal_display
    defsig_fpe_inner.o(.text) refers to defsig_general.o(.text) for __default_signal_display
    defsig_rtred_inner.o(.text) refers to defsig_general.o(.text) for __default_signal_display
    defsig_stak_inner.o(.text) refers to defsig_general.o(.text) for __default_signal_display
    defsig_pvfn_inner.o(.text) refers to defsig_general.o(.text) for __default_signal_display
    defsig_cppl_inner.o(.text) refers to defsig_general.o(.text) for __default_signal_display
    defsig_segv_inner.o(.text) refers to defsig_general.o(.text) for __default_signal_display
    defsig_other.o(.text) refers to defsig_general.o(.text) for __default_signal_display


================================================================================

Removing Unused input sections from the image.

    Removing main.o(.bss), (128 bytes).

1 unused section(s) (total 128 bytes) removed from the image.

================================================================================

Image Symbol Table

    Local Symbols

    Symbol Name                              Value     Ov Type        Size  Object(Section)

    ../../angel/boardlib.s                   0x00000000   Number         0  boardinit3.o ABSOLUTE
    ../../angel/boardlib.s                   0x00000000   Number         0  cpuinit.o ABSOLUTE
    ../../angel/boardlib.s                   0x00000000   Number         0  boardinit1.o ABSOLUTE
    ../../angel/boardlib.s                   0x00000000   Number         0  boardinit2.o ABSOLUTE
    ../../angel/boardlib.s                   0x00000000   Number         0  boardshut.o ABSOLUTE
    ../../angel/kernel.s                     0x00000000   Number         0  kernel.o ABSOLUTE
    ../../angel/rt.s                         0x00000000   Number         0  rt_locale_intlibspace.o ABSOLUTE
    ../../angel/rt.s                         0x00000000   Number         0  rt_locale.o ABSOLUTE
    ../../angel/rt.s                         0x00000000   Number         0  rt_raise.o ABSOLUTE
    ../../angel/rt.s                         0x00000000   Number         0  rt_fp_status_addr_intlibspace.o ABSOLUTE
    ../../angel/rt.s                         0x00000000   Number         0  rt_stackheap_storage.o ABSOLUTE
    ../../angel/rt.s                         0x00000000   Number         0  rt_stackheap_storage_intlibspace.o ABSOLUTE
    ../../angel/rt.s                         0x00000000   Number         0  rt_fp_status_addr.o ABSOLUTE
    ../../angel/startup.s                    0x00000000   Number         0  __main.o ABSOLUTE
    ../../angel/sys.s                        0x00000000   Number         0  use_no_semi.o ABSOLUTE
    ../../angel/sys.s                        0x00000000   Number         0  sys_stackheap_outer.o ABSOLUTE
    ../../angel/sys.s                        0x00000000   Number         0  sys_exit.o ABSOLUTE
    ../../angel/sys.s                        0x00000000   Number         0  libspace.o ABSOLUTE
    ../../angel/sysapp.c                     0x00000000   Number         0  sys_wrch.o ABSOLUTE
    ../../angel/sysapp.c                     0x00000000   Number         0  sys_command.o ABSOLUTE
    ../../armsys.c                           0x00000000   Number         0  no_argv.o ABSOLUTE
    ../../armsys.c                           0x00000000   Number         0  _get_argv.o ABSOLUTE
    ../../armsys.c                           0x00000000   Number         0  lib_init.o ABSOLUTE
    ../../armsys.c                           0x00000000   Number         0  lib_init.o ABSOLUTE
    ../../fpinit.s                           0x00000000   Number         0  fpinit.o ABSOLUTE
    ../../heapalloc.c                        0x00000000   Number         0  hrguard.o ABSOLUTE
    ../../signal.c                           0x00000000   Number         0  defsig_rtmem_outer.o ABSOLUTE
    ../../signal.c                           0x00000000   Number         0  defsig_stak_inner.o ABSOLUTE
    ../../signal.c                           0x00000000   Number         0  defsig_pvfn_inner.o ABSOLUTE
    ../../signal.c                           0x00000000   Number         0  defsig_cppl_inner.o ABSOLUTE
    ../../signal.c                           0x00000000   Number         0  defsig_exit.o ABSOLUTE
    ../../signal.c                           0x00000000   Number         0  defsig_segv_inner.o ABSOLUTE
    ../../signal.c                           0x00000000   Number         0  defsig_fpe_inner.o ABSOLUTE
    ../../signal.c                           0x00000000   Number         0  defsig_other.o ABSOLUTE
    ../../signal.c                           0x00000000   Number         0  defsig_rtmem_inner.o ABSOLUTE
    ../../signal.c                           0x00000000   Number         0  __raise.o ABSOLUTE
    ../../signal.c                           0x00000000   Number         0  defsig_general.o ABSOLUTE
    ../../signal.c                           0x00000000   Number         0  defsig_abrt_inner.o ABSOLUTE
    ../../signal.c                           0x00000000   Number         0  defsig_rtmem_formal.o ABSOLUTE
    ../../signal.c                           0x00000000   Number         0  defsig_rtred_inner.o ABSOLUTE
    ../../signal.s                           0x00000000   Number         0  defsig.o ABSOLUTE
    ../../stdlib.c                           0x00000000   Number         0  exit.o ABSOLUTE
    ../../stkheap.s                          0x00000000   Number         0  heapext.o ABSOLUTE
    ../../stkheap1.s                         0x00000000   Number         0  stkheap1.o ABSOLUTE
    ../../stkheap2.s                         0x00000000   Number         0  stkheap2.o ABSOLUTE
    ..\MK1986BE_HID\startup_MPS.s            0x00000000   Number         0  startup_mps.o ABSOLUTE
    Main.c                                   0x00000000   Number         0  main.o ABSOLUTE
    dc.s                                     0x00000000   Number         0  dc.o ABSOLUTE
    RESET                                    0x08000000   Section      192  startup_mps.o(RESET)
    !!!main                                  0x080000c0   Section        8  __main.o(!!!main)
    .emb_text                                0x080000c8   Section        4  lib_init.o(.emb_text)
    .text                                    0x080000cc   Section      464  main.o(.text)
    .text                                    0x0800029c   Section       56  startup_mps.o(.text)
    .text                                    0x080002d4   Section       38  stkheap2.o(.text)
    .text                                    0x080002fa   Section       62  kernel.o(.text)
    .text                                    0x08000338   Section       74  sys_stackheap_outer.o(.text)
    .text                                    0x08000384   Section       12  rt_stackheap_storage_intlibspace.o(.text)
    .text                                    0x08000390   Section       20  sys_exit.o(.text)
    .text                                    0x080003a4   Section        8  libspace.o(.text)
    .text                                    0x080003ac   Section       12  exit.o(.text)
    .text                                    0x080003b8   Section      192  lib_init.o(.text)
    .text                                    0x08000478   Section       10  boardinit2.o(.text)
    .text                                    0x08000482   Section        8  boardinit3.o(.text)
    .text                                    0x0800048a   Section        2  use_no_semi.o(.text)
    .text                                    0x0800048c   Section       12  rt_locale_intlibspace.o(.text)
    .text                                    0x08000498   Section        2  no_argv.o(.text)
    .text                                    0x0800049c   Section       12  rt_fp_status_addr_intlibspace.o(.text)
    x$fpl$fpinit                             0x080004a8   Section       14  fpinit.o(x$fpl$fpinit)
    .bss                                     0x20000000   Section       96  libspace.o(.bss)
    HEAP                                     0x20000060   Section     1024  startup_mps.o(HEAP)
    Heap_Mem                                 0x20000060   Data        1024  startup_mps.o(HEAP)
    STACK                                    0x20000460   Section     1024  startup_mps.o(STACK)
    Stack_Mem                                0x20000460   Data        1024  startup_mps.o(STACK)
    __initial_sp                             0x20000860   Number         0  startup_mps.o(STACK)

    Global Symbols

    Symbol Name                              Value     Ov Type        Size  Object(Section)

    BuildAttributes$$THM_ISAv4$M$P$D$K$S$PE$A:L22UL41UL21$X:L11$S22US41US21$IEEE1$IW$USESV6$~STKCKD$USESV7$~SHL$OSPACE$EBA8$STANDARDLIB$REQ8$PRES8$EABIv2 0x00000000   Number         0  anon$$obj.o ABSOLUTE
    __ARM_use_no_argv                        0x00000000   Number         0  main.o ABSOLUTE
    __ARM_exceptions_init                     - Undefined Weak Reference
    __Heap_DescSize                           - Undefined Weak Reference
    __alloca_initialize                       - Undefined Weak Reference
    __cpp_initialize__aeabi_                  - Undefined Weak Reference
    __cxa_finalize                            - Undefined Weak Reference
    __scatterload                             - Undefined Weak Reference
    __sigvec_lookup                           - Undefined Weak Reference
    __user_heap_extend                        - Undefined Weak Reference
    _atexit_init                              - Undefined Weak Reference
    _call_atexit_fns                          - Undefined Weak Reference
    _clock_init                               - Undefined Weak Reference
    _fp_trap_init                             - Undefined Weak Reference
    _get_lc_collate                           - Undefined Weak Reference
    _get_lc_ctype                             - Undefined Weak Reference
    _get_lc_monetary                          - Undefined Weak Reference
    _get_lc_numeric                           - Undefined Weak Reference
    _get_lc_time                              - Undefined Weak Reference
    _getenv_init                              - Undefined Weak Reference
    _handle_redirection                       - Undefined Weak Reference
    _init_alloc                               - Undefined Weak Reference
    _init_user_alloc                          - Undefined Weak Reference
    _initio                                   - Undefined Weak Reference
    _rand_init                                - Undefined Weak Reference
    _signal_init                              - Undefined Weak Reference
    _terminate_user_alloc                     - Undefined Weak Reference
    _terminateio                              - Undefined Weak Reference
    __Vectors                                0x08000000   Data           4  startup_mps.o(RESET)
    __main                                   0x080000c1   Thumb Code     8  __main.o(!!!main)
    __ARM_argv_veneer                        0x080000c9   Thumb Code     4  lib_init.o(.emb_text)
    main                                     0x080000cd   Thumb Code   414  main.o(.text)
    Reset_Handler                            0x0800029d   Thumb Code     4  startup_mps.o(.text)
    NMI_Handler                              0x080002a1   Thumb Code     2  startup_mps.o(.text)
    HardFault_Handler                        0x080002a3   Thumb Code     2  startup_mps.o(.text)
    MemManage_Handler                        0x080002a5   Thumb Code     2  startup_mps.o(.text)
    BusFault_Handler                         0x080002a7   Thumb Code     2  startup_mps.o(.text)
    UsageFault_Handler                       0x080002a9   Thumb Code     2  startup_mps.o(.text)
    SVC_Handler                              0x080002ab   Thumb Code     2  startup_mps.o(.text)
    DebugMon_Handler                         0x080002ad   Thumb Code     2  startup_mps.o(.text)
    PendSV_Handler                           0x080002af   Thumb Code     2  startup_mps.o(.text)
    SysTick_Handler                          0x080002b1   Thumb Code     2  startup_mps.o(.text)
    AACI_IRQHandler                          0x080002b3   Thumb Code     0  startup_mps.o(.text)
    CAN_IRQHandler                           0x080002b3   Thumb Code     0  startup_mps.o(.text)
    CHLCD_IRQHandler                         0x080002b3   Thumb Code     0  startup_mps.o(.text)
    CLCD_IRQHandler                          0x080002b3   Thumb Code     0  startup_mps.o(.text)
    ENET_IRQHandler                          0x080002b3   Thumb Code     0  startup_mps.o(.text)
    FLEXRAY_IRQHandler                       0x080002b3   Thumb Code     0  startup_mps.o(.text)
    I2C_IRQHandler                           0x080002b3   Thumb Code     0  startup_mps.o(.text)
    LIN_IRQHandler                           0x080002b3   Thumb Code     0  startup_mps.o(.text)
    MCIA_IRQHandler                          0x080002b3   Thumb Code     0  startup_mps.o(.text)
    MCIB_IRQHandler                          0x080002b3   Thumb Code     0  startup_mps.o(.text)
    RTC_IRQHandler                           0x080002b3   Thumb Code     0  startup_mps.o(.text)
    SPI_IRQHandler                           0x080002b3   Thumb Code     0  startup_mps.o(.text)
    TIM0_IRQHandler                          0x080002b3   Thumb Code     0  startup_mps.o(.text)
    TIM2_IRQHandler                          0x080002b3   Thumb Code     0  startup_mps.o(.text)
    UART0_IRQHandler                         0x080002b3   Thumb Code     0  startup_mps.o(.text)
    UART1_IRQHandler                         0x080002b3   Thumb Code     0  startup_mps.o(.text)
    UART2_IRQHandler                         0x080002b3   Thumb Code     0  startup_mps.o(.text)
    UART3_IRQHandler                         0x080002b3   Thumb Code     0  startup_mps.o(.text)
    USBDC_IRQHandler                         0x080002b3   Thumb Code     0  startup_mps.o(.text)
    USBHC_IRQHandler                         0x080002b3   Thumb Code     0  startup_mps.o(.text)
    WDT_IRQHandler                           0x080002b3   Thumb Code     0  startup_mps.o(.text)
    __user_initial_stackheap                 0x080002b5   Thumb Code     0  startup_mps.o(.text)
    __use_two_region_memory                  0x080002d5   Thumb Code     2  stkheap2.o(.text)
    __rt_stackheap_init                      0x080002d7   Thumb Code    24  stkheap2.o(.text)
    __rt_heap_extend                         0x080002ef   Thumb Code    12  stkheap2.o(.text)
    __rt_entry                               0x080002fb   Thumb Code    36  kernel.o(.text)
    __rt_exit                                0x0800031f   Thumb Code    18  kernel.o(.text)
    __rt_abort                               0x08000331   Thumb Code     8  kernel.o(.text)
    __user_setup_stackheap                   0x08000339   Thumb Code    74  sys_stackheap_outer.o(.text)
    __rt_stackheap_storage                   0x08000385   Thumb Code     6  rt_stackheap_storage_intlibspace.o(.text)
    _sys_exit                                0x08000391   Thumb Code    16  sys_exit.o(.text)
    __user_libspace                          0x080003a5   Thumb Code     4  libspace.o(.text)
    __user_perproc_libspace                  0x080003a5   Thumb Code     0  libspace.o(.text)
    __user_perthread_libspace                0x080003a5   Thumb Code     0  libspace.o(.text)
    exit                                     0x080003ad   Thumb Code    12  exit.o(.text)
    __rt_lib_init                            0x080003b9   Thumb Code   174  lib_init.o(.text)
    __rt_lib_shutdown                        0x08000467   Thumb Code    18  lib_init.o(.text)
    _platform_post_stackheap_init            0x08000479   Thumb Code    10  boardinit2.o(.text)
    _platform_post_lib_init                  0x08000483   Thumb Code     8  boardinit3.o(.text)
    __I_use_semihosting                      0x0800048b   Thumb Code     0  use_no_semi.o(.text)
    __use_no_semihosting_swi                 0x0800048b   Thumb Code     2  use_no_semi.o(.text)
    __rt_locale                              0x0800048d   Thumb Code     6  rt_locale_intlibspace.o(.text)
    __ARM_get_argv                           0x08000499   Thumb Code     2  no_argv.o(.text)
    __rt_fp_status_addr                      0x0800049d   Thumb Code     6  rt_fp_status_addr_intlibspace.o(.text)
    _fp_init                                 0x080004a9   Thumb Code    14  fpinit.o(x$fpl$fpinit)
    __fplib_config_pureend_doubles           0x080004b5   Thumb Code     0  fpinit.o(x$fpl$fpinit)
    __libspace_start                         0x20000000   Data          96  libspace.o(.bss)
    __temporary_stack_top_libspace           0x20000060   Data           0  libspace.o(.bss)


================================================================================

Memory Map of the image

  Image Entry point : 0x080000c1

  Load Region LR_IROM1 (Base: 0x08000000, Size: 0x000004b8, Max: 0x00010000, ABSOLUTE)

    Execution Region ER_IROM1 (Base: 0x08000000, Size: 0x000004b8, Max: 0x00010000, ABSOLUTE)

    Base Addr    Size         Type   Attr      Idx    E Section Name        Object

    0x08000000   0x000000c0   Data   RO           85    RESET               startup_mps.o
    0x080000c0   0x00000008   Code   RO           95  * !!!main             __main.o(c_w.l)
    0x080000c8   0x00000004   Code   RO          116    .emb_text           lib_init.o(c_w.l)
    0x080000cc   0x000001d0   Code   RO            1    .text               main.o
    0x0800029c   0x00000038   Code   RO           86    .text               startup_mps.o
    0x080002d4   0x00000026   Code   RO           93    .text               stkheap2.o(c_w.l)
    0x080002fa   0x0000003e   Code   RO           97    .text               kernel.o(c_w.l)
    0x08000338   0x0000004a   Code   RO          100    .text               sys_stackheap_outer.o(c_w.l)
    0x08000382   0x00000002   PAD
    0x08000384   0x0000000c   Code   RO          105    .text               rt_stackheap_storage_intlibspace.o(c_w.l)
    0x08000390   0x00000014   Code   RO          107    .text               sys_exit.o(c_w.l)
    0x080003a4   0x00000008   Code   RO          109    .text               libspace.o(c_w.l)
    0x080003ac   0x0000000c   Code   RO          112    .text               exit.o(c_w.l)
    0x080003b8   0x000000c0   Code   RO          117    .text               lib_init.o(c_w.l)
    0x08000478   0x0000000a   Code   RO          122    .text               boardinit2.o(c_w.l)
    0x08000482   0x00000008   Code   RO          124    .text               boardinit3.o(c_w.l)
    0x0800048a   0x00000002   Code   RO          128    .text               use_no_semi.o(c_w.l)
    0x0800048c   0x0000000c   Code   RO          133    .text               rt_locale_intlibspace.o(c_w.l)
    0x08000498   0x00000002   Code   RO          139    .text               no_argv.o(c_w.l)
    0x0800049a   0x00000002   PAD
    0x0800049c   0x0000000c   Code   RO          148    .text               rt_fp_status_addr_intlibspace.o(c_w.l)
    0x080004a8   0x0000000e   Code   RO          141    x$fpl$fpinit        fpinit.o(fz_ws.l)
    0x080004b6   0x00000002   PAD
    0x080004b8   0x00000000   Data   RO          188    Region$$Table       anon$$obj.o


    Execution Region RW_IRAM1 (Base: 0x20000000, Size: 0x00000860, Max: 0x00010000, ABSOLUTE, UNINIT)

    Base Addr    Size         Type   Attr      Idx    E Section Name        Object

    0x20000000   0x00000060   Zero   RW          110    .bss                libspace.o(c_w.l)
    0x20000060   0x00000400   Zero   RW           84    HEAP                startup_mps.o
    0x20000460   0x00000400   Zero   RW           83    STACK               startup_mps.o


================================================================================

Image component sizes


      Code (inc. data)   RO Data    RW Data    ZI Data      Debug   Object Name

       464         50          0          0          0       4570   main.o
        56         22        192          0       2048        288   startup_mps.o

    ------------------------------------------------------------------------
       520         72        192          0       2048       4860   Object Totals
         0          0          0          0          0          0   (incl. Generated)
         0          0          0          0          0          2   (incl. Padding)

    ------------------------------------------------------------------------

      Code (inc. data)   RO Data    RW Data    ZI Data      Debug   Library Member Name

         8          0          0          0          0          0   __main.o
        10          0          0          0          0          0   boardinit2.o
         8          0          0          0          0          0   boardinit3.o
        12          0          0          0          0          0   exit.o
        14          0          0          0          0          0   fpinit.o
        62          0          0          0          0          0   kernel.o
       196          0          0          0          0          0   lib_init.o
         8          4          0          0         96          0   libspace.o
         2          0          0          0          0          0   no_argv.o
        12          6          0          0          0          0   rt_fp_status_addr_intlibspace.o
        12          6          0          0          0          0   rt_locale_intlibspace.o
        12          6          0          0          0          0   rt_stackheap_storage_intlibspace.o
        38          0          0          0          0          0   stkheap2.o
        20         10          0          0          0          0   sys_exit.o
        74          0          0          0          0          0   sys_stackheap_outer.o
         2          0          0          0          0          0   use_no_semi.o

    ------------------------------------------------------------------------
       496         32          0          0         96          0   Library Totals
         6          0          0          0          0          0   (incl. Padding)

    ------------------------------------------------------------------------

      Code (inc. data)   RO Data    RW Data    ZI Data      Debug   Library Name

       476         32          0          0         96          0   c_w.l
        14          0          0          0          0          0   fz_ws.l

    ------------------------------------------------------------------------
       496         32          0          0         96          0   Library Totals

    ------------------------------------------------------------------------

================================================================================


      Code (inc. data)   RO Data    RW Data    ZI Data      Debug   

      1016        104        192          0       2144       4860   Grand Totals
      1016        104        192          0       2144       4860   ELF Image Totals
      1016        104        192          0          0          0   ROM Totals

================================================================================

    Total RO  Size (Code + RO Data)                 1208 (   1.18kB)
    Total RW  Size (RW Data + ZI Data)              2144 (   2.09kB)
    Total ROM Size (Code + RO Data + RW Data)       1208 (   1.18kB)

================================================================================

